:020000040000FA
:10000000012803138316033085000030860000307A
:100010008700831287150716FF30860005118512A9
:1000200007173D2207139020C80DC8034810C91BAD
:100030004814C81B6C28481B6C28C81A2028232881
:10004000481A26282928481A2C282D28C8192E286D
:100050003128C819342837283A283A2848196228FC
:100060005D2848195828532848194E284928481906
:1000700044283F280130CA006330CB0071280A3081
:10008000CA005A30CB0071281430CA005030CB005F
:1000900071281E30CA004630CB0071282830CA00B3
:1000A0003C30CB0071283230CA003230CB0071288E
:1000B0003C30CA002830CB0071284630CA001E30C0
:1000C000CB0071285030CA001430CB0071285A3050
:1000D000CA000A30CB0071286330CA000130CB005F
:1000E0007128CA0B7428772807177C2071280713FA
:1000F0007C20CB0B77281328CF01CE014808CC00F9
:1001000090214F08EF2186000515552205114E0854
:10011000EF218600851655228512FF3086000800E3
:10012000871507164B2207120000000000008711F8
:10013000000000000000071688210712882107121E
:10014000882107168821071288210716882107129F
:100150008821071288218316071683128821071E1B
:10016000AF284B2283160712831207128821071229
:100170008821071288210712882107128821071277
:1001800088210712882107128821831607168312F7
:100190008821071EC9284B22831607128312871550
:1001A00000000000000007164B22071200000000AC
:1001B00000008711000000000000071688210712C8
:1001C000882107128821071688210712882107161F
:1001D000882107128821071688214B2283160716CB
:1001E00083124B22C8010000000087154B22071A1A
:1001F000C817000087110000000087154B22071A5E
:100200004817000087110000000087154B22071ACD
:10021000C816000087110000000087154B22071A3E
:100220004816000087110000000087154B22071AAE
:10023000C815000087110000000087154B22071A1F
:100240004815000087110000000087154B22071A8F
:10025000C814000087110000000087154B22071A00
:100260004814000087114B22C901000000008715C7
:100270004B22071AC91700008711000000008715DC
:100280004B22071A4917000087110000000087154C
:100290004B22071AC91600008711000000008715BD
:1002A0004B22071A4916000087110000000087152D
:1002B0004B22071AC915000087110000000087159E
:1002C0004B22071A4915000087110000000087150E
:1002D0004B22071AC914000087110000000087157F
:1002E0004B22071A49140000871183160712831244
:1002F0008715000087110000071600000712000094
:10030000000000000000871500000000071608002C
:10031000000087150000640000008711000008003D
:100320006400CC0B94290800CE0ACE18CE1D9A2961
:10033000CF0ACE01CF18CF1D90290F30CE00CF00AD
:100340000800CD004D18A829A529CD18B129AB2941
:10035000CD18B429AE294D19C329B7294D19C6297D
:10036000BA294D19C929BD294D19CC29C029CD1942
:10037000DF29CF29CD19E129D129CD19E329D329A5
:10038000CD19E529D529CD19E729D729CD19E9298D
:10039000D929CD19EB29DB29CD19ED29DD2911301A
:1003A0000800BD3008005830080038300800B6306A
:1003B00008003230080012300800B9300800103050
:1003C000080030300800FE300800FE300800FE3023
:1003D0000800FE300800FE300800FE300800CD00A6
:1003E0004D18F629F329CD18FF29F929CD18022A2D
:1003F000FC294D19112A052A4D19142A082A4D19CC
:10040000172A0B2A4D191A2A0E2ACD192D2A1D2A10
:10041000CD192F2A1F2ACD19312A212ACD19332A85
:10042000232ACD19352A252ACD19372A272ACD196D
:10043000392A292ACD193B2A2B2A90300800D73097
:100440000800A4300800C4300800CB300800C830D1
:10045000080088300800D530080080300800C0301F
:100460000800EF300800EF300800EF300800EF30F0
:100470000800EF300800EF3008000630C20064309A
:10048000C1006430C0006400C00B442AC10B412A83
:10049000C20B3F2A08000330C1000330C000C00B6C
:1004A0004F2AC10B4D2A64000800FF30C000C00B6A
:0604B000572A6400080059
:02400E00F73F7A
:00000001FF
